:020000040000FA
:060000000219FD0200B32D
:03002B0002008D43
:03005B0002028C12
:030073000200A0E8
:100080000406080C10182030406080A0C0C0D0C00A
:10009000E0C2CF0541E52360021523D0E0D0D03285
:1000A000C2AF53E67F7592FA7593FFC22053917FDA
:1000B000D2AF32C2AF53E6EFC0D0C0E0C0F0D2D36F
:1000C000D2AF5388EFA88AA98C758A00758C00433B
:1000D000881030331FE8C4540FFAE9C454F04AFAC8
:1000E000C3132AFAC3E833F8E933F9E82AFAE93402
:1000F00003FB213D30320FC3E833E933FAE82AFA33
:10010000E93400FB213D303115E875F056A4AAF022
:10011000E975F056A42AFAC5F03400FB213DE875D4
:10012000F02BA4AAF0E975F02BA42AFAC5F034004C
:10013000C313FBEA13FAC3EB13FBEA13FAC3EB9402
:10014000095006C3EB9403501A0522E522700215EC
:1001500022C3E522940A5002417F7552007A007B47
:1001600000414DE522600215223035067C007D04F9
:10017000217DAC31AD32303A04AC33AD34C3EA9CAE
:10018000FAEB9DFB9208AE5EAF5F303A425007201B
:100190003409D234219B303402C234303404AE608E
:1001A000AF61203902B234C3EA33FAEB33FBA20861
:1001B000500AEAF42401FAEBF43400FBC3EA942871
:1001C000FAEB9400FB501478007A007B0021DBA24C
:1001D00008500878007A007B004131E5255403601F
:1001E00019202A16E55BF9EB7007C3E99A4002E98A
:1001F000FAE53CC42AFAEB3400FBEA8EF0A4F9AA33
:10020000F0EB8EF0A42AFAC5F03400FBC3EB13FD2B
:10021000EA13F80FEF146004C3E833F8C3E933EAD4
:1002200033FAEB33FBDFEDEB30E20678FF7AFF7B4E
:10023000038852D230C3E559FC955A4002AC5AC3E8
:10024000EC95525008EC75F004A4FAABF0EAF4F81F
:10025000EBF45403F9C3E89414FAE99400FB500456
:100260007A007B00885489558A568B5775230AD0AB
:10027000F0D0E0D0D053F7DF43F74043E6103275BB
:10028000230AD0F0D0E0D0D043E61032C2AF53A85A
:10029000FEC0D0C0E0D2D3A8F9E55830E10AE5FAB3
:1002A00020E14220E03F41B0E5FA30E13820E0357E
:1002B000C3E55513F8E55413F5FB88FCC3E5571364
:1002C000F8E55613F5E988EA85555853F7BFC3E5B5
:1002D000529401400575530041E5E5532401F5535F
:1002E00050037553FF53F7DFD0E0D0D043A801D2BD
:1002F000AF327901801479038010790A800C791E5D
:1003000080087964800479C880007817E4D5E0FD1E
:10031000D8FAD9F6227A147B7880127A107B8C80F6
:100320000C7A0D7BB480067A0B7BC88000E562D521
:10033000E001227902E4C293D5E0FDD292D5E0FD3E
:10034000C292D5E0FDD293D5E0FDE920E002D29043
:1003500030E002D294E562D5E0FDE920E002C290EF
:1003600030E002C2947496D5E0FDD9C9EAF8D5E030
:10037000FDD8FBDBB8C2932278FF20282879A1E7BB
:100380006023E548601F74FF8548F084853FF030A6
:10039000290375F005A4F8C5F0600278FFC3E8955D
:1003A0005B5002A85B885A22C3E54794E4E5489471
:1003B00000E55A50031461B9046002F55A2275E849
:1003C0009022055CC3E55C9408405330EDF4A8BD71
:1003D000A9BE755C00E9FA79A0E76041EA7006E51C
:1003E0005D6018800CC3E8955D600EE55D500560AA
:1003F0000A1480070460FA8002E55DF55DC3956725
:10040000401B7559C0C394044013755980C39404AC
:10041000400B755940C39404400375590022E559B7
:100420002410500274FFF55922743279A687F0A483
:10043000C5F0A2F733F8C3E895594002A859885B84
:10044000227547007548F022C2AF75C800A8CCA934
:10045000CDAA4130CF010A75C804D2AFAB42AC433C
:1004600088428943C3E89BF8E99C202808F9302C8E
:1004700002A15781B1AD448A44F9EA9DFA6004783B
:10048000FF79FFAE45AF468B458C46A842A943C3D2
:10049000E89EF8E99FF9C3E54813FBE54713FAE83E
:1004A0002AF547E93BF54850067547FF7548FF8137
:1004B000FEAA47AB48AC47AD487E047F02C3EB942D
:1004C00004400D1E1FC3EB940840052029021E1F87
:1004D000C3ED13FDEC13FCDEF7C3EA9CFAEB9DFBC6
:1004E000EF6009C3E913F9E813F8DFF7EA28FAEB3C
:1004F00039FB8A478B4850067BFF8B478B48C3EB01
:1005000094025002D22C3028047F03A1297892E66D
:10051000FFC3E53D948240110FC3E53D94A0400127
:100520000FC3EF940640027F057E02E548C4540FD6
:10053000F9E548C454F0F8E547C4540F28F8C3E877
:100540009EFAE99400FB4009C3EA9401EB94005041
:10055000047A01E4FBA1A3AA47AB48EBC4FEEAC4BA
:10056000540F4EFCC3EA9CFAEB9400FBC3E813C3A0
:1005700013F8EA28FAEB3400FB8A478B48C3EB9464
:10058000024002C22C7802EBC4FE7B00EAC4540F86
:100590004EFAC3EA98FA4005C3940150027A0178F2
:1005A00092E6FF302002A1A3854E92854F93D22080
:1005B00043E680C3E49AF8E49BF9302C02C12EE8AC
:1005C000FAE9FBD3E913FDE813FC884E894FC3EF2A
:1005D00094036037EF20E00CE82CF8E93DF9ECFAE1
:1005E000EDFB8013E828F8E939F9C3E82401F8E9BC
:1005F0003400F97AFF7BFFC3EF9403400E8A508BDF
:1006000051884A894B8C4C8D4DC162885089518AE2
:100610004A8B4B8C4C8D4D3028127550F07551FF24
:10062000754CF0754DFF754EF0754FFFC162E8FADD
:10063000D3E813FC884EC3EF94036020EF20E0075B
:10064000E82CF8ECFAC14EE8282401F87AFFC3EF51
:10065000940340088A50884A8C4CC16288508A4A68
:100660008C4C302002C162753A02D22043E680E50C
:100670002554036034A847A948C3E913F9E813F8DF
:10068000C3E913F9E813F8302804E92440F9C2AFAC
:1006900053E67F759100C3E498F594E499F5957558
:1006A0009104D22043E680D2AF22D2217549007551
:1006B0002000302B03752040800ED2217549007533
:1006C0002040302B0375200078017901202C20E593
:1006D0002554036002C2217914E548C31370010454
:1006E000F8C3941440027814302804781B791B2036
:1006F0002010E549600C302803D53A04D223E1727A
:10070000D16A0549E59B5440B52002E15C302809D7
:1007100008C3E899400118C1EF20210A08C3E899ED
:100720004002C1C8C1EFC221C2AF53E67F7591003C
:10073000302C127594007595F8759104D22043E61B
:1007400080D2AFC1C8E5487EFFC3334005C3334004
:1007500001FEC3E49E759400F595E139C3E5399433
:10076000015002C1C8302102C1C8D802E170C1EFF6
:10077000C223C2AF53E67F75910085509485519591
:10078000759104854A92854B93D22043E680D2AF7F
:10079000E525540360072029020539801030230D18
:1007A000202B0A20210715811581020EB022780026
:1007B0003021027801E53D75F007A4F9E5F028F550
:1007C000F0E9A2F013A2F113A2F213F53DC394785D
:1007D0005003753D78C3E53D953E400BD222C29053
:1007E000C292C29475D57F302002E1E7854C928594
:1007F0004D93D22043E68022203810C2AFC293D25C
:100800009175D54FD2AF759F2001CCC2AFC293D2A4
:100810009575D57CD2AF759F2001CC203811C2AF21
:10082000C29475D573D291D2AF759F300208CCC2F5
:10083000AFC29075D573D295D2AF759F100208CC18
:10084000203810C2AFC291D29575D573D2AF759FC3
:10085000108079C2AFC295D29175D573D2AF759F12
:10086000308069203811C2AFC29275D57CD295D242
:10087000AF759F200208CCC2AFC29275D54FD291FE
:10088000D2AF759F200208CC203810C2AFC295D2DB
:100890009375D57CD2AF759F308031C2AFC291D2F3
:1008A0009375D54FD2AF759F108021203810C2AFFD
:1008B000C29075D54FD293D2AF759F10800EC2AF44
:1008C000C29475D57CD293D2AF759F30C22222C21A
:1008D00090C292C294C291C293C29575D57F22787C
:1008E0008076FF0876FF0876FF0876FF0876FF0817
:1008F00076FF0876090876FF087601788C7601087D
:1009000076FF0876FF0876FF0876FF0876FF087600
:10091000030876FF0876FF0876FF0876250876D06C
:100920000876280876500876040876FF08760208CC
:1009300076FF08767A0876FF08760708760108764B
:10094000FF0876FF08760008760022FA75F00CA4FE
:10095000ABF0EAC333F8740133F9E8C333F8E93391
:10096000F9E8C32BF8E93400F9227888E6C3940348
:10097000D23A5002C23AC238E630E102D238A23846
:1009800092397886E6149000809378A6F67886E609
:10099000F53FC394025003753F02789CE6753EFF15
:1009A000B40203753EA0B40303753E8278A0E6F856
:1009B000600674282409D8FCF5677896E6314B88E0
:1009C000318932789EE6314B883389347897E63125
:1009D0004B8835893611CF223035117A007B007C67
:1009E000FF7D007E00513F8B5F8A5E22303A227885
:1009F00096E6FA7B00789EE6FC7D00C3EA33FAEBCC
:100A000033FBC3EC33FCED33FD7E0A513F8B618A2F
:100A1000607896303A02789EE6FA7B007897E6FC9A
:100A20007D007E00303A10C3EA33FAEB33FBC3ECAF
:100A300033FCED33FD7E0A513F8B5F8A5E2222C379
:100A4000EC9EFCED9400FDC3EC9AFCED9BFDC3EC29
:100A50009423ED940050047C237D00C3EC94FFEDBF
:100A6000940140047CFF7D017BFF0B7A000AEA7051
:100A700009C3EC33FCED33FD416AEC8AF0A4AEF01F
:100A8000ED8AF0A42E947C40E4EAF460DD22D235B5
:100A900031D81202FE1202FE7A007B007C10120294
:100AA000F6E5522AFA74003BFBDCF37C04C3EB133B
:100AB000FBEA13FADCF7FFEB60027FFFC23531D8A7
:100AC0002278A5E6F95403D2867002C286E9540C56
:100AD000D2877002C287E95430D2967002C296E97A
:100AE00054C07000227565007566007597DE7597B5
:100AF000AD7581C043FF8075EF0675A90011CF75F4
:100B0000803F75F1F075A4C075803F75D4FF759076
:100B10000075F27F75A57F75900075D57F75A6016C
:100B200075E34075E202C290C292C294120302D2EF
:100B300091D293D2951202F2C291C293C29511CF73
:100B4000E4F8F6D8FD11DFD1E278988662753001BD
:100B5000C2AF1203061203151202FE12031B120289
:100B6000FE1203211202FE51C1C2AF756500756607
:100B70000078FA79FA308507D9FBD8F7021C0031E2
:100B80006A31D87898866211CF75E4057588117539
:100B90008E0475890975C80475910475D84075D996
:100BA0000875F781759E0375960275DA4275DB420A
:100BB00075A82175E69075F310759B80759D00757D
:100BC000D10C75BC5975BB1075E88075B201120265
:100BD000F2D2AF753C00C230120306C2317522005A
:100BE000120302C3E522940A4024D231C232752294
:100BF00000120302C3E522940A4013D232C23375B5
:100C00002200120302C3E522940A4002D2331202E8
:100C1000F6203003020B69C2AF120315120315123E
:100C20000315D2AF120306303A0281CB1202F678D6
:100C30008CE6C39401500281CBE530C3940150028D
:100C400081CB7565A57566F17F02D23531D8120367
:100C500002C2AFC23531D8C3E552947FD2AF406BE8
:100C60001202F2C2AF120327D2AFDFDE518EC3EF02
:100C70007897F6120306F1C27F0AD23531D81203F3
:100C800002C2AFC23531D8C3E552947FD2AF50E82B
:100C90001202F2C2AF1203151202FA120315D2AFFA
:100CA000DFD8518EEF24037896F6F87997E7C3944E
:100CB000234003985006E824237897F6120306F1A0
:100CC0001C120FF112030231D86169756500756657
:100CD000001203027801303A027805C3E5529840C9
:100CE000028127C2AF120327120327120327D2AFB4
:100CF000120306753000E4F537F5380537E537F4AB
:100D0000703E0538789AE6781914601278321460CB
:100D10000D787D14600878FA146003753800C3E517
:100D20003898401C11CF1202F215387537007899A7
:100D30008662C2AF120327D2AF789886621203028E
:100D40001202FAE523700261697801C3E552984006
:100D5000AA120302E5237003020B69C2AF11CFE4AC
:100D6000D2AFE4F55CF524F525F53D755C0812027B
:100D7000F21203BE30EDFDA8BDA9BEE97001F888EE
:100D80005D1203C2755C08C2AF7559FF1204298554
:100D90005B59855B5AD2AF303A07C238303402D241
:100DA00038D228753900118811AB12044112044859
:100DB0001204411204481204411206BA1207AE127C
:100DC00007F81204481206AA202C03120378302CCC
:100DD000031203A81207AE111B1204481206BA121E
:100DE00007AE11401204481206AA1207AE11631290
:100DF00004481206BA1207AE11881204481203BE44
:100E00001206AA1207AE11AB1203C2120448302810
:100E100027855B5979187A0CC3E53999400EC228A9
:100E2000D2298A3B855B59855B5A800CC3E5529475
:100E3000014003020DB9C1B830291C202B19E53B34
:100E4000147006C229D22AA1B9F53BC3E552940118
:100E50004003020DB98061753C0078FA79A4E7601F
:100E6000027803C3E55398504FE523604B303A179F
:100E7000203805203407800F303402800A202B07E9
:100E8000D22B855B59A1E778F0302B05855B59782B
:100E900020C3E548985003020DB9302B1BC22BC26A
:100EA00038303402D238D229753B12855B59A1B94A
:100EB000053CE5526002C1BB753C00C2AF11CF7565
:100EC0002400752500D2AF12030211CF78A4E6608A
:100ED00006D291D293D295C3E53C94044002616955
:100EE00081F6901A0D7820F155E520B4550AA3F14A
:100EF00055E520B4AA02800611DFF11C801D901A6E
:100F00000378807B0AF155A308DBFA901A0F788CDE
:100F10007B1AF155A308DBFA901A2922C2AFF19887
:100F2000F175901A007410F15AA37403F15AA37466
:100F300021F15A901A0378807B0AF159A308DBFA51
:100F4000901A0F788C7B1AF159A308DBFAF1ABF1F8
:100F500089901A2922E493F622E6438F01538FFDEC
:100F6000FFC3E583941C400122EF8565B78566B712
:100F7000F0538FFE22438F02438F018565B785664C
:100F8000B7901A0DF0538FFC22901A0D7455F15A38
:100F9000901A0E74AAF15A227A3079D07820901AD9
:100FA00040F155E520F709A3DAF7227A3079D0909D
:100FB0001A40E7F15A09A3DAF9227C05120306DC8C
:100FC000FB22C2AF12031512031B120321120327C7
:100FD0001202FA12031512031B1203211203271225
:100FE00002FA12031512031B120321120327D2AFB8
:100FF00022C2AF12032712032112031B1203151280
:1010000002FA12032712032112031B120315120204
:10101000FA12032712032112031B120315D2AF2267
:1019FD00020AE5100321FFFFFFFFFFFF09FF01FFB3
:101A0D0055AA01FFFFFFFFFF03FFFFFF25D0285061
:0D1A1D0004FF02FF7AFF0701FFFF0000FF3A
:101A400023455F4C5F32302320202020202020209F
:101A500023424C48454C492445464D3842313023B9
:101A60002020202020202020202020202020202076
:101C0000C2AFC2D37597DE7597AD7581C075A90057
:101C100043FF80752438752503B1DB7529A5752A26
:101C2000F143F12053A4DFD28575D4FF75E3407DE5
:101C3000FA780379E67C10752200752300901DE880
:101C40007B0675249875250130850281482085081A
:101C5000D8FBD9F9DCF781BA308508D8FBD9F9DC93
:101C6000F781BAB19BE493A3C39A6004DDC381BA40
:101C7000DBDBB18D600281317B08E493FAA3B16EA6
:101C8000DBF87A30B16E752200752300B18DEAFC65
:101C9000EBFDC3ED94FE400EB18D8A278B28ED300D
:101CA000E0048A828B83B18D7AC270D8C3ED94FE32
:101CB000601950CEBD0029EC600F7520007521FF22
:101CC000752900752A000200008100A827A92808AC
:101CD00009D804D90281DDB191EAF281D10D81A642
:101CE000C3ED94035051EDA2E092007AC5C3E582A2
:101CF0009400E583941C508C200010438F02438F86
:101D0000018529B7852AB7F0300027A827A9280818
:101D100009438F01538FFDD804D902A132C3E58353
:101D2000941C4003A3A117E28529B7852AB7F0A325
:101D3000A117538FFC81827AC1BD030CE493A3FAEF
:101D4000B152DCF8B14A81828184AA22AB23B16E00
:101D5000EBFAEA6222752608C3E52313F523E52290
:101D600013F52250066323A0632201D526EAB1DBD6
:101D7000B1DB75260AEAF4200102D285300102C2E5
:101D800085B1DBC3134002C201D526EB22B191EA33
:101D9000FB208502A191308502A196752608AE240C
:101DA000AF25C3EF13FFEE13FEB1DFB1DBC3EA13C0
:101DB0003085024480FA30E703632201C3E5231330
:101DC000F523E52213F52250066323A0632201D5F3
:101DD00026D9E52265236523F52222AE24AF250E00
:101DE0000FDEFEDFFCD20122424C48656C693437BD
:061DF0003163E8B10601B9
:00000001FF
